:020000040000FA
:0A000000700ED36E9B8CC1D166D048
:08001800036ED8CF02F0FACF0D
:1000200004F09EBA63D08A6A936AF29400000000DA
:1000300000000000FF0E896E0000000000000000BC
:10004000FF0E936E8A6EF9500550F92636D02ED0E9
:1000500026D01ED016D00ED006D0056A120E896E9C
:100060001E1C936E32D00E0E056E030E896E1D1C83
:10007000936E2BD00C0E056E130E896E1C1C936EA6
:1000800024D00A0E056E000E896E1B1C936E1DD0C7
:10009000080E056E100E896E1A1C936E16D0060E91
:1000A000056E020E896E191C936E0FD0040E056E3C
:1000B000010E896E181C936E08D0AFEC00F0020E92
:1000C000056E110E896E171C936E035002C0D8FF87
:1000D00004C0FAFF1000630ECF6EBF0ECE6E9E906E
:1000E000397039B011003A663A0611009E9AABA2F7
:1000F00005D0AB98AE50AE50AE50AB88ABA402D09A
:10010000AE50E3D7D624436E3FB4DFD73FB005D01F
:10011000AE50CC0ADAE13F80D8D73FB207D0AE501C
:10012000F00A01E0D2D73F82416ACFD710EE80F0CB
:100130004150AECFE3FF412A100E4162C6D73F8443
:10014000416A3F903F92F29E010EFC6E560EFD6E8C
:10015000080EFE6E000EFF6EF950F28E1000216642
:1001600011D007C017F008C018F009C019F00AC074
:100170001AF00BC01BF00CC01CF00DC01DF00EC01F
:100180001EF01200202E08D01FC020F0232E04D015
:1001900021C023F0226622062250205CD8B0E1D78D
:1001A0000FC017F010C018F011C019F012C01AF0EB
:1001B00013C01BF014C01CF015C01DF016C01EF0BB
:1001C000120007C00FF008C010F009C011F00AC0FB
:1001D00012F00BC013F00CC014F00DC015F00EC0DF
:1001E00016F01FC022F01FC020F021C023F0120023
:10030000F9264FEF02F07AEF02F0C6EF02F00EEF9F
:1003100003F037EF03F03EEF03F056EF03F05DEF2D
:1003200003F064EF03F06BEF03F072EF03F079EF8B
:1003300003F080EF03F0C2EF02F087EF03F08EEFDF
:1003400003F095EF03F09CEF03F0A3EF03F0AAEFA7
:1003500003F0B1EF03F0B8EF03F0BFEF03F0C6EF27
:1003600003F0CDEF03F0D4EF03F0DBEF03F0E2EFA7
:1003700003F0E9EF03F003EF04F00AEF04F011EFEC
:1003800004F018EF04F01FEF04F000EE00F0EE5060
:10039000002600B0012AEAA0FAD700EE00F00066BD
:1003A00002D0450E006E016602D0300E016EA7EC41
:1003B00004F0FF0E896E8A6E936E0F0EC16E6C0E86
:1003C000926E898E000E216E0C0E1F6E426A416A7B
:1003D000080EB86E460EAF6E100EB06E040EAC6E08
:1003E000C00ED56ED66ACD6A000ECD6E630ECF6E8E
:1003F000BF0ECE6ECD80F26A9D6AA06A9E6AF06AD8
:10040000800EF16E010E9F6ED08E9D80E00EF26E1A
:10041000900EAB6EFF0E076E086E096E0A6E0B6EC5
:100420000C6E0D6E0E6EE1EC00F0FA0EDEEC04F0D8
:10043000C4EC04F0640EDEEC04F0216A29C02AF05A
:1004400028C029F027C028F0210E3C6E000ECFEC0A
:1004500004F0276E27503FBA09D0286201D0F4D7A4
:10046000296201D0F1D72A6201D0EED73F9A070E58
:100470003C6E010ECFEC04F0066E230E3C6E070EB0
:10048000CFEC04F02B6EC4EC04F037BEC2EF02F0E8
:10049000F950030EFA6E2750040DF35031D7460E73
:1004A0003C6E140ECFEC04F0066E050E3C6E010E91
:1004B000CFEC04F0216EE1EC00F0ADEC04F000C0F4
:1004C00007F001C008F0ADEC04F000C009F001C075
:1004D0000AF0ADEC04F000C00BF001C00CF0ADEC84
:1004E00004F000C00DF001C00EF026EC04F0062E62
:1004F000E4D7A3D7040E216EE1EC00F0FF0E076EE7
:10050000086E096E0A6E0B6E0C6E0D6E0E6EC80EC6
:10051000DEEC04F0040E3C6E010ECFEC04F0216E14
:1005200000EE07F0ADEC04F0070E0014E926ADEC88
:1005300004F0070E0114256EFE0E266E255204E00F
:1005400026462650252EFCD7E1EC00F0EFCF26F012
:10055000EF162650EF6204D0002AD8B0012AE0D767
:1005600026EC04F00766DCD70866DAD70966D8D728
:100570000A66D6D70B66D4D70C66D2D70D66D0D70D
:100580000E66CED7640EDEEC04F057D7640EDEECB8
:1005900004F0040E3C6E010ECFEC04F0216E00EE70
:1005A00007F0ADEC04F0070E0014E926ADEC04F002
:1005B000070E0114256E010E266E2552D8B404D004
:1005C00026462650252EFCD7E1EC00F0EFCF26F092
:1005D000EF122650EF6204D0002AD8B0012ADFD7EC
:1005E00026EC04F0FF0E0718DAE1FF0E0818D7E139
:1005F000FF0E0918D4E1FF0E0A18D1E1FF0E0B1807
:10060000CEE1FF0E0C18CBE1FF0E0D18C8E1FF0E76
:100610000E18C5E1C80EDEEC04F00FD73C0E3C6EA0
:100620000F0ECFEC04F0066E100E3C6E070ECFECF2
:1006300004F02B6E00EE07F0ADEC04F0070E001492
:10064000E926ADEC04F0070E0114256E010E266EAE
:100650002552D8B404D026462650252EFCD7EF6E5E
:100660002B50DEEC04F0EF6A062EE4D7E6D60B0E34
:10067000336E000E326E020EE2EF04F0060E3C6E98
:10068000010ECFEC04F0216E26EC04F0FF0E076E95
:10069000086E096E0A6E0B6E0C6E0D6E0E6E26ECF9
:1006A00004F0C4EC04F0062EEFD7C7D60B0E336E61
:1006B000180E326E050EE2EF04F00B0E336E480E8C
:1006C000326E070EE2EF04F00B0E336E880E326EC0
:1006D000050EE2EF04F00B0E336EB80E326E050E0F
:1006E000E2EF04F00B0E336EE80E326E020EE2EF14
:1006F00004F00C0E336E000E326E080EE2EF04F0C2
:100700000C0E336E480E326E090EE2EF04F00C0E42
:10071000336E980E326E050EE2EF04F00C0E336E5F
:10072000C80E326E040EE2EF04F00D0E336E000EB2
:10073000326E040EE2EF04F00D0E336E200E326EB8
:10074000050EE2EF04F00D0E336E500E326E070E02
:10075000E2EF04F00C0E336EF00E326E010EE2EF9B
:1007600004F00D0E336E900E326E080EE2EF04F0C0
:100770000D0E336E900E326E020EE2EF04F00D0E8F
:10078000336EF00E326E010EE2EF04F00E0E336E99
:10079000000E326E090EE2EF04F00E0E336E500EB4
:1007A000326E010EE2EF04F00E0E336E600E326E0A
:1007B000010EE2EF04F00E0E336E700E326E050E77
:1007C000E2EF04F00E0E336EA00E326E010EE2EF79
:1007D00004F0190E3C6E0F0ECFEC04F0216E060EE5
:1007E0001F6EE1EC00F0FF0E076E086E096E0A6ED8
:1007F0000B6E0C6E0D6E0E6E26EC04F00C0E1F6E62
:10080000E1EC00F01AD60E0E336EB00E326E010E11
:10081000E2EF04F00E0E336EC00E326E050EE2EF04
:1008200004F00F0E336E000E326E040EE2EF04F091
:100830000F0E336E280E326E040EE2EF04F00F0E30
:10084000336E500E326E030EE2EF04F02266FED7D6
:10085000E1EC00F012003F8C9D9800EE80F0EECFAE
:1008600024F0EECF25F096EC04F0426E446EEECF0D
:1008700024F0EECF25F096EC04F02C6E44263F0ECB
:100880002C6052D0EECF24F0EECF25F096EC04F0A1
:100890002D6E4426EECF24F0EECF25F096EC04F03A
:1008A0002E6E4426EECF24F0EECF25F096EC04F029
:1008B0002F6E4426EECF24F0EECF25F096EC04F018
:1008C000306E4426EECF24F0EECF25F096EC04F007
:1008D000316E4426EECF24F0EECF25F096EC04F0F6
:1008E0003F94441821E12CC027F02DC02BF02EC0DE
:1008F00006F02FC001F030C000F0379E31BE378EB9
:10090000C4EC04F042B007D03F8EFF0E286E296E73
:100910002A6E3F8A92D542A006D0D6CF01F043C0BE
:1009200000F03F9E8AD5FF003F9487D52430010B0D
:1009300024B6020924BA040924BE080925B2100904
:1009400025B6200925BA400925BE8009120000EE0F
:1009500002F0EE6AE9AEFDD71200016604D03FAEA8
:10096000D6CF01F0FAD7006602D0450E006E0134F2
:100970000118E836013A0038E8460118013A010B3F
:100980000036001A01361200076A086A096A0A6A04
:100990000B6A0C6A0D6A0E6AE1EC00F012003B6E05
:1009A000DCDF00C03EF03BC03DF03E4E05D03D2AAE
:1009B0003C503D64FAD7F7D73D5012003A6E3A6684
:1009C000FED71200366E070E3C6E020ECFEC04F01E
:1009D000066E216609D0060E3C6E010ECFEC04F0C7
:1009E000216E21500808066E346A00C035F0C4EC50
:1009F00004F035B20BD0345016EC05F026EC04F0C0
:100A0000342A36503464F7D735B00BD036C034F0C2
:100A1000345016EC05F026EC04F03406FF0E346278
:100A2000F7D7346A062EE5D71DEF02F033C0F7FF83
:100A3000080DF3503224F66E0900F538076E0900F0
:100A4000F538086E0900F538096E0900F5380A6EA8
:100A50000900F5380B6E0900F5380C6E0900F53801
:0A0A60000D6E0800F5380E6E12004E
:100B0000FF0000000000001000FF000000000010C7
:100B10000000FF0000000010000F000000000010A7
:100B20000000F00000000010F000000000000010C5
:100B300000F000000000001000000F000000001096
:100B40000F00000000000010000000000000001076
:100B500018181800000000103C3C3C000060001019
:100B60003C3C3C66666600103C3C3CFFFFFF0010CE
:100B70007E7E7EFFFFFF00107E7E7EFFFFFFFFD3A5
:100B8000FFFFFFFFFFFFFFD3000060000F003000FA
:100B900060000000F000C0000060000000F000C035
:100BA00000000600000F00030600000F0000030015
:100BB000000600F000000C00400000000000C00033
:100BC00000400000000000C0000002000000000320
:100BD00002000000000003000002000000000C0002
:100BE00000004000000030000081000000000CC048
:100BF0000000810000003003810000000000C300FD
:100C000000010000000000000002000000000000E1
:100C100000040000000000000008000000000000C8
:100C200000000000000000100010000000000000A4
:100C30000020000000000000004000000000000054
:100C40000080000000000000000000000000000024
:100C5000010001000000010103000303000303037E
:100C60000700070F000F03030F000F3F003F07436C
:100C70000FFF0F3F003F07531FFF1FFF00FF0FD362
:100C80003FFF3FFFC3FF0FD37FFF7FFFFFFF9FD3D8
:100C9000FFFFFFFFFFFFFFD3F0FFF0C0FFC0F890A2
:100CA000F0F0FF00FCFCE0D2FFF00F03C0FF81D3A7
:100CB0000FFF0F3F003F07530F0FFFFF03031F11ED
:100CC000FF0FF0FC3F007E108181810000000000DA
:100CD0000000000000005582000000111188000093
:100CE0000000008888110000000000000000AA41F8
:100CF000FFFFFF000000FFC3FFFFFF000000000038
:100D0000181818000000000024242400000000002F
:100D1000424242000000000081818100000000008A
:100D2000FFFFFF00000000107E7E7E00000000102C
:100D3000BDBDBD0000000010DBDBDB0000000010CB
:100D4000E7E7E70000000010FFFFFF0000000000E1
:100D500000000001180100000000000118016101FD
:100D60008100810118016101810081011801F303F3
:100D7000810081099909F303810081999999F3030D
:100D8000810081999999FFC3818181999999FFC3C4
:100D90000081000000000000004200000000000090
:100DA0000024000000000000001800000000000007
:100DB00000000000000000101800180000000010E3
:100DC0003C003C00000000107E007E00000000108F
:100DD000FF00FF00000000102400240CC30C0000E2
:100DE000002424300CC30000242400C33030000051
:100DF0000000000000000010818181000000000060
:100E000000000000000000000001000000000000E1
:100E10000003000000000C00010780F801001E0024
:100E2000070FE0FC03003F000F0FF0FF0F003F1023
:100E30003F1FFCFF3F037F11FF3FFFFF7F077F1135
:100E4000FF7FFFFFFFFFFF13FFFFFFFFFFFFFFD34A
:100E5000F00F0FF0F00FCC130FF0F00F0FF033D0B6
:100E6000F00F0F000000CC130FF0F000000033D0A3
:100E70000000100000000000100000000000000052
:100E8000001000000000000000000800000000004A
:100E90000800000000000000000800000000000042
:100EA0000408200000002100201004000000400180
:100EB000A5A5A500000000105A5A5A000000000025
:100EC000FFF0FFFFFFFFFFD3FFFF0FFFFFFFFFD389
:100ED0000FFFFFFFFFFFFFD3FF0FFFFFFFFFFFD35A
:100EE000FFFFF0FFFFFFFFD3F0FFFFFFFFFFFFD388
:100F00000000008888110000000000444422000016
:100F100024242400000000000000002222440000DD
:100F20000000001111880000000000000000001007
:100F300018181800000000103C3C3C000000001095
:100F40003C3C3C66666600103C3C3CFFFFFF0010EA
:100F500000E00000000000000000070000000000AA
:100F60000700000000000000000700000000000073
:081000000000000000000000E8
:020000040030CA
:06000100081E1E0E08811E
:0600080003C003E0034009
:00000001FF
